:020000020000FC
:100000001CC935C20000000023C000004DC1000023
:10001000000050C1000000000000000002030406C0
:10002000080C101820304060800002030406080C01
:10003000101820304080FF000406080C10182030F3
:10004000406080A0C00005050D050D0602030302F7
:100050004FB662FD20C070FF1AC165FDFAC057FEA1
:1000600001C00994C0919700C395C0939700C5E063
:10007000C519B8F3D0919700CD1B98F3C8E7089441
:1000800083FDC795C4BDC52DCC2321F4C0E083FDFD
:10009000C0E8C4BD07C171FF03C0909891989398C0
:1000A000C52D089483FDC795C4BDC09399006B7F8F
:1000B000C52DCF3F09F441C0C0919800C395C093AE
:1000C000980070FF35C09098919893984FBE1895FE
:1000D0007860C091A000CC2391F0C0919800CA959F
:1000E000D091A000CD1B58F0777FC0919800D0919F
:1000F0009F00CD1B08F41CC02092980019C0909856
:1001000091989398C5E0CA95F1F7C0917500CA958A
:10011000C2FD09C0C1FD05C095FF949A95FD959A51
:100120000EC0979A0CC095FF959A95FD949A07C0BA
:100130009098919893984FBE1895209299004FBE31
:100140001895A5C0552021F095FF909A95FD939A9A
:1001500091989DC0552009F0919A95FF939895FD2F
:10016000909895C0552021F095FF939A95FD909A0F
:1001700095FF909895FD93988AC095FF959895FD69
:10018000949895FF949895FD9598C5E0CA95F1F7D8
:10019000552021F095FF909A95FD939A919877C0FC
:1001A00095FF959895FD94989798C5E0CA95F1F7B5
:1001B000552021F095FF909A95FD939A919867C0EC
:1001C000979895FF959895FD9498C5E0CA95F1F795
:1001D000552009F0919A95FF939895FD909857C0F6
:1001E000979895FF949895FD9598C5E0CA95F1F775
:1001F000552009F0919A95FF939895FD909847C0E6
:1002000095FF949895FD95989798C5E0CA95F1F754
:10021000552021F095FF939A95FD909A95FF90981F
:1002200095FD939834C095FF949895FD959895FF0A
:10023000959895FD9498C5E0CA95F1F7552021F061
:1002400095FF939A95FD909A95FF909895FD9398B8
:100250001EC082FF1CC0C0917500C2FD0BC0C1FD55
:1002600011C095FF959895FD949895FF949895FDEC
:1002700095980DC0C1FDF5CF95FF959895FD949883
:10028000979805C0979895FF949895FD9598C52DDA
:10029000C095089483FDC795C4BDC0939900209272
:1002A000970064604FBE18954FB6C0E1C8BF6E7F1F
:1002B0004FBE18953FB68F7EABB7A074A211806178
:1002C000A0E0ABBFA9B7AE7FA9BF7894A0916600AC
:1002D000AA2349F0A92FAF7151F1A0916600AA9508
:1002E000A093660024C040E050E0A0B396FDA09526
:1002F000A2FD4FEF96FFA3E096FDA2E0A5BFAA27BF
:10030000A064AABF8D7FA0B396FDA095A2FD5FEF6C
:10031000451749F7A8E161FDA0936600A92FAF71C9
:1003200019F0A8E1A093660040938D008160A09130
:100330006700AA2331F0A0916700AA95A0936700F7
:1003400007C0A92FAF7121F08061AA27A064AABFBE
:1003500080FF48C0A0918D004A2F8E7FA92FAF71DA
:10036000C1F0403F08F040EFA42FA295AF704A0FB4
:100370005091B000533069F0A695A69550FD01C08C
:10038000A69552FD03C0A41B4A2F03C04A0F08F4D0
:100390004FEFA09196004A1708F44A2F409361004E
:1003A00071FF08C0A091610050919200A51710F054
:1003B00050936100A091610040916300A41B70F014
:1003C0004091CF00A40B50F0A0916300A40FA09324
:1003D000630040F4AFEFA093630004C0A0916100FC
:1003E000A093630040916300A09192004A1708F027
:1003F0004A2F542EA52DA03408F06860A09160000B
:10040000A395A093600051F0F894A9B7A160A9BF8B
:1004100084FF02C0A0E4ABBF3FBE189541E05091FD
:100420006600552331F0A92FAF7119F45A955093F6
:100430006600A0918D00A13018F0209290000DC0B0
:100440002092910020929A00A0919000AF5FA0931B
:10045000900018F0AFEFA0939000F894A9B7A160B6
:10046000A9BF84FF02C0A0E4ABBF3FBE18953FB652
:100470004CB55DB58F7EABB7A074A2118061A0E0D2
:10048000ABBFA9B7AE7FA9BF789481FD26C096FF08
:10049000A2E096FDA3E0A5BF8260A0B396FDA09563
:1004A000A2FF05C0409364005093650033C196FFDE
:1004B000A3E096FDA2E0A5BFAA27A064AABF8D7FF6
:1004C000A92FAF7109F417C140E0A0B396FDA09524
:1004D000A2FD11C140938D0004C196FFA3E096FDDB
:1004E000A2E0A5BF8D7F61FF6BC096FFA2E096FDE5
:1004F000A3E0A5BFAA27A064AABF8260409388009A
:1005000050938900A09086004A19B09087005B093B
:10051000BB24A2E0EA2EA22C483CA0E05A0730F40B
:10052000A0E1BA2EE22CAAE0AA2E27C04836A1E00C
:100530005A0730F4A8E0BA2EE22CAFE0AA2E1DC074
:10054000403DA2E05A0730F4A4E0BA2EE22CAEE11E
:10055000AA2E13C0403AA5E05A0730F4A2E0BA2E02
:10056000E22CACE3AA2E09C04839A8E05A0728F4C7
:10057000A1E0BA2EE22CA8E7AA2EC42EA0918A00F0
:10058000CA1AD52EA0918B00DA0ADD202AF4AFEF2B
:10059000C094D094CA1ADA0A20928C00CA14DE04DD
:1005A00018F4A1E0A0938C0040938A0050938B0034
:1005B00040918800509189004093860050938700B5
:1005C000A09164004A1BA09165005A0B94FD7CC069
:1005D00093FD7AC092FD76C05695479591FD72C005
:1005E0005695479590FD6EC0D52EC42ED694C794CF
:1005F00061FD0CC0AC2DAC51AD2DA24008F07BC00C
:10060000DD2021F4AC2DA85C08F475C0A0E0EA2E32
:1006100097FD08C0E090C200A091B400A33011F48F
:10062000E090CA00AAEFEA0EF22CF21CCE18DF0806
:100630004FB74170A091B400A330A9F4442329F02E
:1006400095FD11C0F894906204C095FF0CC0F89419
:100650009F7D90989198939895989798949871FD0C
:1006600001C060687894442369F0A091B400A3307D
:1006700031F4AFEFC094D094CA1ADA0A03C040E054
:1006800050E022C0A091B400A33049F4CC0CDD1C92
:10069000A5E0CA1AD20818F4A0E0CA2ED22CAFEFF7
:1006A000CA16D20418F04FEF50E00EC0F090A70029
:1006B000CF9C412D000C441F50E008F012C04FEFBA
:1006C00050E00FC05695479594FF07C0552309F099
:1006D0004FEFA42FA6954A0F521D4F3F520508F029
:1006E0004FEF40938D00816061FF05C0AFE1A095A1
:1006F000A923AB299A2FA8E1A0936600A92FAF7177
:1007000019F4AAE0A093660061FD04C0A92FAF719F
:1007100009F08F7EA6E0A0936700A92FAF7119F4AE
:10072000AAE0A0936700F894A9B7A160A9BF84FFCD
:1007300002C0A0E4ABBF3FBE189511E00AC013E0B1
:1007400008C01AE006C01EE104C014E602C018EC9E
:1007500000C005E1BB27BA95F1F70A95D9F71A95BC
:10076000C1F708952AE338E709C020E33CE806C052
:100770002AE234EB03C025E238EC00C0652CB1E07E
:100780005B2E12E095FD9F7D95FF9062BB279798A9
:10079000BA95F1F7552009F0919ABA95F1F7919829
:1007A000BA95F1F7979ABA95F1F7552021F095FF90
:1007B000909A95FD939AB091A800BA95F1F795FF9C
:1007C000909895FD9398B7E8BA95F1F71A95D1F6F8
:1007D000022FB22FBA95F1F70A95D9F73A9571F62B
:1007E0009798562C0895221B39E0001F3A9509F47A
:1007F0000895221F211B18F4210F8894F6CF089426
:10080000F4CF622C722CB0E08894B395221F331F72
:10081000E0F7379527958894912E802E020B130BC5
:1008200010F4192D082D10F4889401C00894661C4A
:10083000771CBA9571F7172D062D0895322D1123C7
:100840002AF43A9500951095031B130BF894029F18
:10085000712C002D129F912C802C7894780C172DE0
:10086000921C292DB4E06B2E2695179507956A9456
:10087000D9F7332321F000951095031B130B08952E
:10088000089566FF21C010917400169500917300C1
:100890000795B0917700B01B0B2FB0917800B10B8A
:1008A0001B2F28F40038BFEF1B0740F009C00F379B
:1008B000120508F405C00FE710E002C000E81FEFC2
:1008C00000937C0010937D00089566FF39C000916D
:1008D0007C00B09179000B0F10917D00B0917A00EF
:1008E0001B1F20E030917D0033230AF42A95B0913C
:1008F0007B002B1F1AF4203F40F00AC02F3008F471
:1009000007C00FEF1FEF2FE003C000E010E020EF63
:1009100030916300B09192003B1718F4332331F00B
:1009200009C0B0917D00BB235AF004C0B0917D0096
:10093000BB2332F40093790010937A0020937B005C
:10094000089566FF2FC02091CD0000917C00000F1C
:1009500010917D00111F72DF11232AF40038BFEFC0
:100960001B0740F009C00F37120508F405C00FE758
:1009700010E002C000E81FEF002352F0B0916200C7
:10098000B01B0B2F18F0013008F00AC001E008C0BE
:1009900000950F5FB09162000B0F08F001C00FEFE0
:1009A00000937E00089566FF2DC02091CE00009137
:1009B0007A0010917B0042DF11232AF40130BFEF4F
:1009C0001B0740F009C00F3F120508F405C00FEFE8
:1009D00010E002C001E01FEF112352F0B0917E0041
:1009E000B01B0B2F18F0013008F00AC000E008C05F
:1009F00000950F5FB0917E000B0F08F001C00FEF64
:100A00000093630008950FEF677FB72FB670E9F486
:100A10006860B0917400B83008F0677FB0917400DE
:100A2000A1F00FEF10917400DEDEF894B091700029
:100A30000B9F112D002D7894112309F00FEFB09129
:100A400095000B1710F40091950000939400089501
:100A50006FC0DDD274FFB7E074FDB7E0B068B0647A
:100A6000B7B9B6B1B068B064B6B967DE74FFB7E0C5
:100A700074FDB7E0B068B064B7B9B6B1B068B0643F
:100A8000B6B9B6B1B6FDFDCF04B115B1B6B1BF77F9
:100A9000B6B902D325E62093A30030E03093A4003A
:100AA000732E7694622E6694620E731E262D372D59
:100AB0000217130778F08090A300B5E6B80DB09345
:100AC000A3008090A400B0E0B81DB093A400260D50
:100AD000371DEECF8090A3009090A4001091A40049
:100AE00016950091A300079516950795B091A30060
:100AF000B00FB093A100B091A400B11FB093A200B9
:100B000023E0169507952A95E1F72091AF002A95E5
:100B100029F42092A3002092A4000AC02A9521F073
:100B2000800E911E2A95E1F78092A3009092A40076
:100B300008952091AF00B6B1B6FDFBCF04B115B159
:100B4000B6B1BF77B6B9B091A500B395B093A50083
:100B5000B83060F12092A500B091CC00BB2321F108
:100B6000112329F0B091A600BF3F61F009C0B091F8
:100B7000A6000B1739F020F4BB2321F0BA9502C070
:100B8000B395E1F300919200B093A600B03050F419
:100B900000ECB03038F400E8B03020F400E4B030BD
:100BA00008F400E0009392007F7E0895B0919200D7
:100BB000B39511F0B0939200B091A500B73009F44D
:100BC0007061089502E3F894B091D0000B9F012D5D
:100BD000000C001F7894B09192000B1710F0009158
:100BE00092000093610000936300502E00939500E3
:100BF000089520927300B8E0B09374000895209196
:100C0000800030918100F8940CB51DB5200F311F84
:100C10003BBD2ABD6160B0E1B8BF789420917100FE
:100C2000309172000093710010937200021B130B3D
:100C30002091730030917400622E732EB4E08B2EDD
:100C4000B2E09B2EB0917400B43010F08A949A9464
:100C5000B83010F08A949A94769467948A94E1F765
:100C600026193709992021F0169507959A94E1F7EE
:100C7000200F311F209373003093740008F0089503
:100C8000BFEFB0937300B093740008952091820079
:100C900030918300F8940CB51DB5020F131F1BBDD6
:100CA0000ABD6160B0E1B8BF7894089560FDFECFE1
:100CB000EDDF0895B091BE0000916E00023808F09B
:100CC000B395003A08F0B395B63008F0B5E09B2E26
:100CD000BCE08B2EB0917400B33030F483948394D5
:100CE00082FF02C083948394B23030F4839483945F
:100CF00082FF02C08394839471FF03C0B3E09B2EF4
:100D0000822C109174000091730024E016950795D1
:100D10002A95E1F70819120928F0B02FB250B12F27
:100D2000B20910F402E010E0312F202F712E602E56
:100D300076946794B92DB330E9F0B0FD05C0060D87
:100D4000171D262D372D06C0000F111F0250120946
:100D500022E030E0B92DB33068F020938400309366
:100D60008500009380001093810060928200709251
:100D700083000895009384001093850020938000E1
:100D8000309381006092820070928300089560FD2C
:100D9000FECF20918200220F30918300331FB72FA6
:100DA000B67021F02091730030917400F8940CB566
:100DB0001DB5020F131F1BBD0ABD6160B0E1B8BFB6
:100DC0007894089560612092760020E004C060610C
:100DD0002092760020E2B72FB67009F06F7E7894EB
:100DE00060FD05C0B0917600BB2309F0089501E0D5
:100DF00063FF0AC0B0917400B33008F002E0B09114
:100E00007400B63008F003E071FF01C006E060FD39
:100E100006C0B0917600BB2311F0789408951AE0D3
:100E200083FF1AE0789400000000F89462FD03C08C
:100E300014E183FF14E171FF01C018E7B4B53091EC
:100E40009900B31BB10B18F3B0917600B395B09332
:100E50007600B5E03B2F6B2E722CB8B1B072B21792
:100E600009F073943A95C9F77394761488F464FF83
:100E7000B2CF6F7E3CB56DB47090730080907400FB
:100E8000370D681C6BBC3ABD6160B0E1B8BFA3CF41
:100E900064FDA1CF0A9509F0BACF7894089571FF47
:100EA0000AC0B0916D00B395B0936D0060FD0CC0A9
:100EB00020926D0009C060FD07C064FD05C067FD9C
:100EC00003C0BF91BF915EC408952091840030910A
:100ED0008500F8940CB51DB5020F131F1BBD0ABD8C
:100EE0006160B0E1B8BF78940895EFDF00E063FF80
:100EF00003C064FF01C001E0F89410916E00B7E0F8
:100F00001B9F212D102D7894200F2695179526953F
:100F100017952695179510936E00183718F4B8E7B3
:100F2000B0936E0000916E00B0916F000B1720F02F
:100F3000606290989198939860FDFECF0895F89420
:100F400095989798949882FF07C0E0E0F1E073FFCE
:100F500003C0BEE1BA95F1F795FF959A95FD949A75
:100F6000B2E0B093750089C0F89495FF939895FD11
:100F7000909882FF0DC0E0EFF0E073FF0BC09798F0
:100F800095FF949895FD9598BEE1BA95F1F702C04A
:100F9000EAEAF0E062FF03C0552009F0919AB3E05D
:100FA000B09375006AC0F89495989798949882FFCA
:100FB00007C0E0EEF0E073FF03C0BEE1BA95F1F7C1
:100FC00095FF949A95FD959AB4E0B093750055C03D
:100FD000F894919882FF0DC0E0EDF0E073FF0BC034
:100FE00095FF959895FD94989798BEE1BA95F1F77D
:100FF00002C0E2EAF0E062FF06C0552021F095FF52
:10100000909A95FD939AB5E0B093750036C0F89428
:1010100095989798949882FF07C0EDEBF0E073FFE6
:1010200003C0BEE1BA95F1F7979AB6E0B0937500A8
:1010300024C0F89495FF909895FD939882FF10C076
:10104000E3E1F1E073FF0EC095FF959895FD94984C
:1010500095FF949895FD9598BEE1BA95F1F702C079
:10106000E2EBF0E062FF06C0552021F095FF939A75
:1010700095FD909AB1E0B093750067FF0AC00CD05F
:10108000BEE1BA95F1F7B5E0BA95F1F7959A979A5E
:10109000949A6F7D7894089521EA30E0F901909850
:1010A000919893989598979894986B7F0895ACEA47
:1010B000B0E00FEF0D930D930D930D9303E00D939F
:1010C00004E00D930AE00D9301E00D9301E00D9310
:1010D00001E00D93A8EBB0E001E00D930FEF0D934D
:1010E0000D930FEF0D930D930D9303E00D9306E019
:1010F0000D930FEF0D930D9305E20D9300ED0D93FE
:101100000AEF0D930AEF0D9304E00D930DE00D939C
:1011100001E00D9300E00D930AE70D930FEF0D939F
:1011200001E00D9308952091BF0009E011E0223005
:1011300011F405E011E0233011F405E012E0243051
:1011400011F405E013E0253011F409E017E0263032
:1011500011F400E010E000939F001093A000209194
:10116000B3008B7F777FB091B400B33019F09F7DCF
:10117000B1FD90629F7BB091B500B1FD9064B22F3C
:10118000B23011F0886001C0877F0895ECE1F0E093
:101190000091AC000A95E00FF21DB491B093CD0020
:1011A0000091AD000A95E00FF21DB491B093CE000E
:1011B00073DF0895EAE2F0E00091C7000A95E00FBE
:1011C000F21DB491B093CF0067DF0895E8E3F0E03B
:1011D0000091B2000A95E00FF21DB491B093D000D7
:1011E0005BDF08950895B091C8000FEF1CE0B230A6
:1011F00011F400EA1AE0B33011F402E815E00093AC
:101200006F0010937000089508952091C2003091EE
:10121000C30097FF02C020E03FEFB32FB21B6B2E3D
:10122000B25810F4B2E86B2E00E00395609EB12D29
:10123000B058D8F30093A7000895F894E3E0F0E0E5
:10124000B9E0B7BFB491B078C1F3F894A895B1B53F
:10125000B861B1BDB0E0B1BDB4E0BEBFBFE5BDBFD8
:101260001BDFB0E0B8BBB0E1B7BBB0E0B5BBB0E0EE
:10127000B4BBB0E0B2BBBBEBB1BB2224A0E0B0E09A
:101280002D92AA31E9F7A0E6B0E00FEF2D920A9572
:10129000E9F70DDF97D247DF79DF8CDF97DFA2DF39
:1012A000A2DFB2DFB2DF0091C4000093A800F4DE39
:1012B000B2E0B3BFB2E0BEBDB2E0B5BDF89447DA6C
:1012C00051DA41DA52DA3FDA53DA3DDA06D33FDA5D
:1012D0003EDA3BDAB1E5B8BFB9BFB0B7B860B0BF6E
:1012E000B6B1B460B6B929DA7894B2DBB0E4BBBF6A
:1012F000BB27B064BABF8D7F2ADAB1E0B093690032
:10130000626025E0B0918C00BB2309F425E017DA78
:10131000B0918D00B230A8F3B92FBF7100918F004A
:1013200000938E00B0938F00B01759F72A9551F7AC
:101330006D7F96FFB3E096FDB2E0B5BFBB27B0640A
:10134000BABF8D7F02DAFBD902E0B92FBF7109F471
:1013500000E0B0918D00B017B0F3F89403DA02DA30
:1013600001DA7894F4D920927F00B091B400B330C0
:1013700009F472C0E4D9B091B800B13008F46CC07F
:10138000B0916900B13008F467C0B92FBF71C1F0E6
:10139000B0918D00BF3F08F45FC0F894ECD9789409
:1013A000D4D9B0918D00B130C0F7F894DBD9C9D948
:1013B000D9D97894CAD9B0918D00BF3FB0F3BFC2DC
:1013C000B8E09B2E9068F89420DF7894BED9F8940A
:1013D0009F771BDF80908D00B0918D00BF37789490
:1013E00008F442C0AAD9F894C6D978949A9451F7CF
:1013F000B82DB550B093C300AAD9F89410D272D2C8
:101400007894BAE09B2E9068F894FFDE78949DD98A
:10141000F8949F77FADE80908D00B0918D00BF37F1
:10142000789478F78AD9F8949DD98BD99BD97894F8
:101430009A9449F7B82DBB5FB093C20088D9F8944D
:10144000EED15FD2789481D9F894DFDE7894B091B0
:101450008D00BF3FC0F373C200918D00B0917F003B
:101460000B1710F000937F0070D901E0B091B40029
:10147000B35009F405E0B0918D00B01708F075CFB6
:10148000F89479D978D977D9789461D9209269007C
:1014900020926A0020926B00B0916A00B395B093DD
:1014A0006A00BF3F69F5B0916B00B395B0936B00D4
:1014B000B091C60009E1BA9559F002E3BA9541F03E
:1014C0000DE7BA9529F00AEFBA9511F020926B005A
:1014D000B0916B00B017A0F0B0916B00BA95B093CB
:1014E0006B00B4EBB0936A00B091C500B093A80054
:1014F000F89441D97894B091C400B093A80025D94C
:1015000020D9B0916600BB2321F4B92FBF7109F433
:10151000F7CEB0918D00B63008F4BECFB091B400D4
:10152000B35009F012D9B0916600BB2309F4E8CE9C
:10153000F894B2DD20926100209262002092630054
:10154000522C7894B091B100B0939600209277001D
:10155000209278002092790020927A0020927B00DD
:101560002092A50060E070E020926E0042DBB8E0BF
:10157000B093A5007061E1D874FFB7E074FDB7E0E7
:10158000B068B064B7B9B6B1B068B064B6B9B6B156
:10159000B6FDFDCF04B115B1B6B1BF77B6B9112311
:1015A00009F00FEF0093A600C4DAB8E0B093A500ED
:1015B00070618090B300B2E0B093B300B4DD80926C
:1015C000B300F894BFEFB0939200FCDAB0916100E1
:1015D000B0939200B0939300B09394007894B1E0EC
:1015E000B0936100B09363005B2EB0939B00B09109
:1015F0009100B0939A007160726020926D0007DDD7
:1016000018DDFDDAF6DA56DB04C08DDD2092A50088
:101610007F7E95FFB2E095FDB4E0B068B064B7B9E5
:10162000D6DB3DDC52DC2CD960DC89DCE8DA3EDB41
:1016300041DBADDBB3E0B068B064B7B9C3DB2FDC2E
:1016400044DC1FD9E0D951DC8FDCD9DA2FDB32DB67
:101650009EDB95FFB4E095FDB2E0B068B064B7B929
:10166000B6DB1DDC32DC31D940DC9DDCC8DA1EDBA8
:1016700021DB8DDB95FFB2E095FDB4E0B068B0648E
:10168000B7B9A0DB0CDC21DC5CD92FDCA1DCB7DA3C
:101690000DDB10DB7CDBB3E0B068B064B7B997DB7F
:1016A000FEDB13DC80D921DCB2DCA9DAFFDA02DB55
:1016B0006EDB95FFB4E095FDB2E0B068B064B7B9F9
:1016C00081DB74FFB7E074FDB7E0B068B064B7B910
:1016D000B6B1B068B064B6B9E2DBF7DB06DCA9DC12
:1016E0008EDAE4DAE7DA25DA52DB71FF25C067FD2E
:1016F00023C0B0919500B0939200B0939300B09145
:101700009100B0939A00B1E0B0939B0014E624E1FD
:10171000B0916D00B11750F07D7F746020936C0024
:10172000BFEFB0939200B093930006C0B0918D00CC
:10173000B13008F06ECF26C072FF10C067FD0EC03A
:10174000B0916C00BA9511F47B7F5FCFB0936C00C1
:10175000B0918D00B13008F05CCF14C0B091900012
:10176000B23880F4B92FBF7121F4B0916600BB2369
:1017700049F0B091740000EF67FF01C000E6B017B8
:1017800008F447CFF89488DC8090B300B2E0B093BF
:10179000B300C9DC8092B300209261002092620005
:1017A00020926300522C209296007E7F7894C5D7B9
:1017B00073DCB92FBF7129F4B0916600BB2309F423
:1017C0009FCD66CEEDE0F0E023D00A3509F01BC0D6
:1017D000EEE0F0E01DD0053A09F015C03AE0ACEAC1
:1017E000B0E0E3E0F0E014D00D9331963A95D9F7EC
:1017F00035E1A8EBB0E0EFE0F0E00AD00D933196D0
:101800003A95D9F702C053DC0AD0E4E2F0E008953B
:10181000E199FECFEEBBFFBBE09A0DB308951ED059
:101820003AE0ACEAB0E0E3E0F0E00D910FD03196A1
:101830003A95D9F735E1A8EBB0E0EFE0F0E00D9193
:1018400005D031963A95D9F712D00895E199FECF97
:101850000DBBEEBBFFBBE29AE19A0895EDE0F0E02C
:101860000FEFF4DFEEE0F0E00FEFF0DF0895EDE0D2
:10187000F0E00AE5EBDFEEE0F0E005EAE7DF0895EF
:101880003091A9000091AA00313011F40093B0000A
:10189000323011F40093B100333011F40093B200F0
:1018A000343011F40093BE00353011F40093C700BA
:1018B000363011F40093BF00373011F40093B300B9
:1018C000383011F40093C800393011F40093B4009B
:1018D0003A3011F40093B500089525E038D72A95E1
:1018E000E9F708953FD741D743D745D72AD73AD705
:1018F0003CD73ED740D725D735D737D739D73BD771
:10190000089539D735D731D72DD71BD734D730D70E
:101910002CD728D716D72FD72BD727D723D708953B
:101920008090A9009090AA001DD71CD71BD709D77B
:101930008A94D1F720D705D79A94E1F70895F894BF
:10194000D1DF7894CADFC9DFB1E0B093A900B1E07C
:10195000B093AA002092AB00F894E2DF7894B5E04F
:101960006B2E70908D00F3D6B0918D007B16C9F769
:10197000B13018F0BF3F40F107C082DFF8944FDF6D
:10198000B1DFB8E0B1BDA9DF6A9459F7B091AB00FF
:10199000B395B093AB00B33008F4DECF9EDFB091C7
:1019A000AA00B395B093AA00F894B091A900BA9593
:1019B000E6E4F0E0EB0FF21D049178940395B0910A
:1019C000AA00B01708F4C6CF88DF87DFB091A9005E
:1019D000B395B093A900B091A900BB3008F4B7CF7C
:0C19E00066DBF8941CDFB8E0B1BD77DFD7
:00000001FF
